BL51 BANKED LINKER/LOCATER V5.03                                                        10/24/2007  13:51:43  PAGE 1


BL51 BANKED LINKER/LOCATER V5.03, INVOKED BY:
C:\KEIL\C51\BIN\BL51.EXE .\Out\main.obj, .\Code\EEPROM.LIB TO .\Out\EEPROM TEST PRINT (.\EEPROM TEST.m51) RAMSIZE (256)


MEMORY MODEL: SMALL


INPUT MODULES INCLUDED:
  .\Out\main.obj (MAIN)
  .\Code\EEPROM.LIB (EEPROM)
  C:\KEIL\C51\LIB\C51S.LIB (?C_STARTUP)
  C:\KEIL\C51\LIB\C51S.LIB (?C?COPY)


LINK MAP OF MODULE:  .\Out\EEPROM TEST (MAIN)


            TYPE    BASE      LENGTH    RELOCATION   SEGMENT NAME
            -----------------------------------------------------

            * * * * * * *   D A T A   M E M O R Y   * * * * * * *
            REG     0000H     0008H     ABSOLUTE     "REG BANK 0"
            DATA    0008H     0020H     UNIT         _DATA_GROUP_
            DATA    0028H     0013H     UNIT         ?DT?_EEPROM_BYTE_CHANGE?EEPROM
            IDATA   003BH     0009H     UNIT         _IDATA_GROUP_
            IDATA   0044H     0006H     UNIT         ?ID?_EEPROM_BYTE_CHANGE?EEPROM
            IDATA   004AH     0001H     UNIT         ?STACK

            * * * * * * *  X D A T A   M E M O R Y  * * * * * * *
                    0000H     0100H                  *** GAP ***
            XDATA   0100H     0200H     ABSOLUTE     

            * * * * * * *   C O D E   M E M O R Y   * * * * * * *
            CODE    0000H     0003H     ABSOLUTE     
            CODE    0003H     0182H     UNIT         ?PR?_EEPROM_BYTE_CHANGE_ERAM?EEPROM
            CODE    0185H     0155H     UNIT         ?PR?_EEPROM_BYTE_CHANGE?EEPROM
            CODE    02DAH     00F6H     UNIT         ?C?LIB_CODE
            CODE    03D0H     00DEH     UNIT         ?PR?MAIN?MAIN
            CODE    04AEH     0027H     UNIT         ?PR?_EEPROM_BYTE_PROGRAM?EEPROM
            CODE    04D5H     001EH     UNIT         ?CO?MAIN
            CODE    04F3H     001EH     UNIT         ?PR?_EEPROM_PAGE_CLEAN?EEPROM
            CODE    0511H     000FH     UNIT         ?PR?EEPROM_ENABLE?EEPROM
            CODE    0520H     000CH     UNIT         ?C_C51STARTUP
            CODE    052CH     0006H     UNIT         ?PR?EEPROM_DISABLE?EEPROM



OVERLAY MAP OF MODULE:   .\Out\EEPROM TEST (MAIN)


SEGMENT                                       DATA_GROUP          IDATA_GROUP
  +--> CALLED SEGMENT                       START    LENGTH     START    LENGTH
-------------------------------------------------------------------------------
?C_C51STARTUP                               -----    -----      -----    -----
  +--> ?PR?MAIN?MAIN

?PR?MAIN?MAIN                               0008H    000FH      003BH    0003H
  +--> ?CO?MAIN
BL51 BANKED LINKER/LOCATER V5.03                                                      10/24/2007  13:51:43  PAGE 2


  +--> ?PR?_EEPROM_PAGE_CLEAN?EEPROM
  +--> ?PR?_EEPROM_BYTE_PROGRAM?EEPROM
  +--> ?PR?_EEPROM_BYTE_CHANGE_ERAM?EEPROM

?PR?_EEPROM_PAGE_CLEAN?EEPROM               0017H    0004H      -----    -----
  +--> ?PR?EEPROM_ENABLE?EEPROM
  +--> ?PR?EEPROM_DISABLE?EEPROM

?PR?_EEPROM_BYTE_PROGRAM?EEPROM             0017H    0002H      -----    -----
  +--> ?PR?EEPROM_ENABLE?EEPROM
  +--> ?PR?EEPROM_DISABLE?EEPROM

?PR?_EEPROM_BYTE_CHANGE_ERAM?EEPROM         0017H    0011H      003EH    0006H
  +--> ?PR?EEPROM_ENABLE?EEPROM
  +--> ?PR?EEPROM_DISABLE?EEPROM



SYMBOL TABLE OF MODULE:  .\Out\EEPROM TEST (MAIN)

  VALUE           TYPE          NAME
  ----------------------------------

  -------         MODULE        MAIN
  C:0000H         SYMBOL        _ICE_DUMMY_
  D:0090H         PUBLIC        P1
  D:00A0H         PUBLIC        P2
  D:00B0H         PUBLIC        P3
  D:00A8H         PUBLIC        IE
  C:04E4H         PUBLIC        TB
  C:04E9H         PUBLIC        TC
  D:00B8H         PUBLIC        IP
  C:03D0H         PUBLIC        main
  D:0098H         PUBLIC        SCON
  D:0088H         PUBLIC        TCON
  C:04D5H         SYMBOL        _?ix1000
  C:04DAH         SYMBOL        _?ix1001
  D:00C8H         PUBLIC        T2CON
  D:00D0H         PUBLIC        PSW
  -------         PROC          MAIN
  -------         DO            
  D:0008H         SYMBOL        TB
  D:000DH         SYMBOL        TC
  I:003BH         SYMBOL        address
  I:003DH         SYMBOL        i
  -------         ENDDO         
  C:03D0H         LINE#         24
  C:03D0H         LINE#         25
  C:03D0H         LINE#         39
  C:03E3H         LINE#         40
  C:03F6H         LINE#         44
  C:03FDH         LINE#         46
  C:0404H         LINE#         47
  C:0410H         LINE#         48
  C:0410H         LINE#         49
  C:0420H         LINE#         50
  C:0428H         LINE#         51
BL51 BANKED LINKER/LOCATER V5.03                                                      10/24/2007  13:51:43  PAGE 3


  C:042DH         LINE#         53
  C:0434H         LINE#         54
  C:0440H         LINE#         55
  C:0440H         LINE#         56
  C:0450H         LINE#         57
  C:0458H         LINE#         58
  C:045DH         LINE#         61
  C:0470H         LINE#         64
  C:0483H         LINE#         65
  C:0496H         LINE#         66
  C:04A9H         LINE#         80
  C:04A9H         LINE#         81
  C:04A9H         LINE#         82
  C:04ACH         LINE#         83
  -------         ENDPROC       MAIN
  -------         ENDMOD        MAIN

  -------         MODULE        EEPROM
  C:0000H         SYMBOL        _ICE_DUMMY_
  D:0090H         PUBLIC        P1
  D:00B0H         PUBLIC        P3
  B:00A8H.7       PUBLIC        EA
  D:00A8H         PUBLIC        IE
  D:00B8H         PUBLIC        IP
  D:00F7H         PUBLIC        ISPC
  D:0098H         PUBLIC        SCON
  D:0088H         PUBLIC        TCON
  D:00F4H         PUBLIC        ISPFAH
  X:0100H         PUBLIC        rambuffer
  D:00F5H         PUBLIC        ISPFAL
  C:04F3H         PUBLIC        _EEPROM_Page_Clean
  C:0003H         PUBLIC        _EEPROM_Byte_change_Eram
  C:04AEH         PUBLIC        _EEPROM_Byte_Program
  C:052CH         PUBLIC        EEPROM_Disable
  D:00C8H         PUBLIC        T2CON
  C:0185H         PUBLIC        _EEPROM_Byte_change
  C:0511H         PUBLIC        EEPROM_Enable
  D:00F6H         PUBLIC        ISPFD
  D:00BFH         PUBLIC        SCONF
  D:00D0H         PUBLIC        PSW
  -------         PROC          EEPROM_ENABLE
  C:0511H         LINE#         23
  C:0511H         LINE#         24
  C:0511H         LINE#         25
  C:0514H         LINE#         26
  C:0517H         LINE#         27
  C:051AH         LINE#         28
  C:051DH         LINE#         29
  C:051FH         LINE#         30
  -------         ENDPROC       EEPROM_ENABLE
  -------         PROC          EEPROM_DISABLE
  C:052CH         LINE#         34
  C:052CH         LINE#         35
  C:052CH         LINE#         37
  C:052FH         LINE#         38
  C:0531H         LINE#         39
  -------         ENDPROC       EEPROM_DISABLE
BL51 BANKED LINKER/LOCATER V5.03                                                      10/24/2007  13:51:43  PAGE 4


  -------         PROC          _EEPROM_PAGE_CLEAN
  D:0006H         SYMBOL        eFlashAddr
  -------         DO            
  D:0017H         SYMBOL        CodePTR
  D:0019H         SYMBOL        FlashAddr
  -------         ENDDO         
  C:04F3H         LINE#         78
  C:04F3H         LINE#         79
  C:04F3H         LINE#         83
  C:04F7H         LINE#         85
  C:04FAH         LINE#         87
  C:0502H         LINE#         88
  C:0505H         LINE#         89
  C:0508H         LINE#         91
  C:050BH         LINE#         92
  C:050EH         LINE#         94
  -------         ENDPROC       _EEPROM_PAGE_CLEAN
  -------         PROC          _EEPROM_BYTE_PROGRAM
  D:0006H         SYMBOL        eFlashAddr
  D:0005H         SYMBOL        eFlashData
  -------         DO            
  D:0082H         SYMBOL        CodePTR
  D:0017H         SYMBOL        FlashAddr
  -------         ENDDO         
  C:04AEH         LINE#         101
  C:04AEH         LINE#         102
  C:04AEH         LINE#         106
  C:04B2H         LINE#         108
  C:04B5H         LINE#         110
  C:04BDH         LINE#         111
  C:04C0H         LINE#         112
  C:04C3H         LINE#         113
  C:04C5H         LINE#         115
  C:04CAH         LINE#         116
  C:04CAH         LINE#         117
  C:04CDH         LINE#         118
  C:04CDH         LINE#         119
  C:04CFH         LINE#         121
  C:04CFH         LINE#         122
  C:04D2H         LINE#         123
  C:04D2H         LINE#         125
  -------         ENDPROC       _EEPROM_BYTE_PROGRAM
  -------         PROC          _EEPROM_BYTE_CHANGE
  D:0028H         SYMBOL        eFlashAddrCustomer1
  D:002AH         SYMBOL        eFlashAddrBuffer1
  D:002CH         SYMBOL        eFlashAddr1
  D:002EH         SYMBOL        eFlashData1
  D:002FH         SYMBOL        Number1
  -------         DO            
  I:0044H         SYMBOL        i
  D:0031H         SYMBOL        CodePTR
  D:0006H         SYMBOL        CodePTR1
  D:0033H         SYMBOL        CodePTR2
  I:0046H         SYMBOL        CusAddrH
  I:0047H         SYMBOL        CusAddrL
  I:0048H         SYMBOL        ChangeAddrH
  I:0049H         SYMBOL        ChangeAddrL
BL51 BANKED LINKER/LOCATER V5.03                                                      10/24/2007  13:51:43  PAGE 5


  D:0035H         SYMBOL        FlashAddr1
  D:0037H         SYMBOL        FlashAddrCustomer1
  D:0039H         SYMBOL        FlashAddrBuffer1
  -------         ENDDO         
  C:0185H         LINE#         133
  C:0191H         LINE#         134
  C:0191H         LINE#         151
  C:0197H         LINE#         153
  C:019DH         LINE#         155
  C:01A3H         LINE#         157
  C:01ABH         LINE#         159
  C:01AFH         LINE#         161
  C:01B7H         LINE#         163
  C:01BBH         LINE#         165
  C:01BEH         LINE#         172
  C:01C1H         LINE#         177
  C:01C4H         LINE#         179
  C:01C7H         LINE#         180
  C:01CAH         LINE#         181
  C:01CDH         LINE#         185
  C:01DFH         LINE#         186
  C:01DFH         LINE#         188
  C:01E6H         LINE#         190
  C:01EEH         LINE#         192
  C:01F5H         LINE#         194
  C:01F8H         LINE#         196
  C:01FBH         LINE#         198
  C:01FFH         LINE#         200
  C:0202H         LINE#         204
  C:0221H         LINE#         205
  C:0221H         LINE#         206
  C:0224H         LINE#         207
  C:0224H         LINE#         208
  C:0226H         LINE#         210
  C:0226H         LINE#         211
  C:022EH         LINE#         212
  C:0231H         LINE#         213
  C:0231H         LINE#         215
  C:023DH         LINE#         217
  C:0246H         LINE#         219
  C:0250H         LINE#         228
  C:0256H         LINE#         229
  C:025CH         LINE#         230
  C:0262H         LINE#         231
  C:026AH         LINE#         232
  C:026EH         LINE#         233
  C:0276H         LINE#         237
  C:0279H         LINE#         238
  C:027CH         LINE#         240
  C:027FH         LINE#         241
  C:0282H         LINE#         242
  C:0294H         LINE#         243
  C:0294H         LINE#         249
  C:029BH         LINE#         250
  C:029FH         LINE#         251
  C:02A6H         LINE#         252
  C:02A9H         LINE#         253
BL51 BANKED LINKER/LOCATER V5.03                                                      10/24/2007  13:51:43  PAGE 6


  C:02ACH         LINE#         266
  C:02B6H         LINE#         267
  C:02B9H         LINE#         271
  C:02C5H         LINE#         272
  C:02CEH         LINE#         274
  C:02D7H         LINE#         276
  -------         ENDPROC       _EEPROM_BYTE_CHANGE
  -------         PROC          _EEPROM_BYTE_CHANGE_ERAM
  D:0017H         SYMBOL        eFlashAddrCustomer
  D:0019H         SYMBOL        eFlashAddr
  D:0001H         SYMBOL        eFlashData
  D:001CH         SYMBOL        Number
  -------         DO            
  I:003EH         SYMBOL        i
  D:001EH         SYMBOL        CodePTR
  D:0006H         SYMBOL        CodePTR1
  D:0020H         SYMBOL        CodePTR2
  I:0040H         SYMBOL        CusAddrH
  I:0041H         SYMBOL        CusAddrL
  I:0042H         SYMBOL        ChangeAddrH
  I:0043H         SYMBOL        ChangeAddrL
  D:0022H         SYMBOL        FlashAddr
  D:0024H         SYMBOL        FlashAddrCustomer
  D:0026H         SYMBOL        FlashAddrBuffer
  -------         ENDDO         
  C:0003H         LINE#         284
  C:000DH         LINE#         285
  C:000DH         LINE#         301
  C:0013H         LINE#         303
  C:0019H         LINE#         305
  C:001FH         LINE#         307
  C:0027H         LINE#         308
  C:002BH         LINE#         309
  C:0033H         LINE#         310
  C:0037H         LINE#         311
  C:003AH         LINE#         312
  C:003DH         LINE#         328
  C:0052H         LINE#         329
  C:0052H         LINE#         330
  C:0059H         LINE#         331
  C:0061H         LINE#         332
  C:0068H         LINE#         335
  C:006BH         LINE#         336
  C:006EH         LINE#         337
  C:0072H         LINE#         338
  C:0075H         LINE#         341
  C:0094H         LINE#         342
  C:0094H         LINE#         343
  C:00A5H         LINE#         346
  C:00A7H         LINE#         348
  C:00A7H         LINE#         349
  C:00BFH         LINE#         352
  C:00BFH         LINE#         353
  C:00CBH         LINE#         354
  C:00D4H         LINE#         356
  C:00DFH         LINE#         359
  C:00E5H         LINE#         360
BL51 BANKED LINKER/LOCATER V5.03                                                      10/24/2007  13:51:43  PAGE 7


  C:00EBH         LINE#         361
  C:00F1H         LINE#         362
  C:00F9H         LINE#         363
  C:00FDH         LINE#         364
  C:0105H         LINE#         366
  C:0108H         LINE#         367
  C:010BH         LINE#         369
  C:010EH         LINE#         371
  C:0111H         LINE#         372
  C:0114H         LINE#         373
  C:0129H         LINE#         374
  C:0129H         LINE#         375
  C:0130H         LINE#         376
  C:0134H         LINE#         377
  C:013BH         LINE#         378
  C:013EH         LINE#         379
  C:0141H         LINE#         392
  C:0155H         LINE#         393
  C:0162H         LINE#         394
  C:0165H         LINE#         396
  C:0171H         LINE#         397
  C:017AH         LINE#         399
  C:0182H         LINE#         401
  -------         ENDPROC       _EEPROM_BYTE_CHANGE_ERAM
  -------         ENDMOD        EEPROM

  -------         MODULE        ?C?COPY
  C:03AAH         PUBLIC        ?C?COPY
  -------         ENDMOD        ?C?COPY

*** WARNING L16: UNCALLED SEGMENT, IGNORED FOR OVERLAY PROCESS
    SEGMENT: ?PR?_EEPROM_BYTE_CHANGE?EEPROM

Program Size: data=75.0 xdata=512 code=1330
LINK/LOCATE RUN COMPLETE.  1 WARNING(S),  0 ERROR(S)
